:100100007B027D017F011201BE7B027D807F021296
:1001100001BE7B027D407F021201BE7B027D207FFB
:10012000021201BE7B027D107F021201BE7D017FA3
:10013000011202767D807F021202767D407F0212DC
:1001400002767D207F021202767D107F02120276F7
:10015000E4FFFEE4F508F5090509E5097002050864
:10016000B4E8F5E508B403F00FBF00010EEF6464D6
:100170004E70E07D017F011202377D807F02120206
:10018000377D407F021202377D207F021202377DC9
:10019000107F02120237E4FEFFC3EF9484EE940353
:1001A000508BE4F508F5090509E50970020508B466
:0E01B000E8F5E508B403F00FBF00010E80DB98
:10026200E4F59AF591F5A1F59BF592F5A2F5A0F5C5
:0402720090F5802261
:1001BE00EF701CEB7006EDF4529A529BBB0107EDEB
:1001CE00F4529AED429BEB64027043ED429A22EF99
:1001DE006401701CEB7006EDF452915292BB010754
:1001EE00EDF45291ED4292EB64027022ED429122B7
:1001FE00EF64027019EB7006EDF452A152A2BB012E
:0F020E0007EDF452A1ED42A2BB0203ED42A12283
:10028900EF70028D80BF01028D90BF02028DA02206
:10027600EF7003ED4280BF0103ED4290BF0203ED34
:0302860042A02271
:10023700EF7004EDF45280BF0104EDF45290BF0259
:0602470004EDF452A022B8
:0F029900EF7003AF8022BF0103AF9022AFA0220E
:10024D00EF7005E5805DFF22BF0105E5905DFF22A2
:05025D00E5A05DFF2299
:0300000002021DDC
:10021D0078FFE4F6D8FD9000007F007E01E4F0A3A6
:0A022D00DFFCDEFA75810902010012
:00000001FF
